:030000000219FDE5
:03000B000200AA46
:03002B0002019C33
:03005B000203524B
:030073000203384D
:1000800002030406080C10182030406080040608A3
:100090000C10182030406080A0C000070F1F3F0DDB
:1000A0000D0403060D0503030202C2AF306308C24C
:1000B00063857C8AD2AF32C0D0C0E0206227E525BC
:1000C0006002E473E525F4C3334009758A00D26306
:1000D000F57C01D6F58A758B00758D00D262D0E073
:1000E000D0D0D2AF32C3E526334009758A00D2633F
:1000F000F57C01F6F58AC262E526F4603C306803BF
:10010000207213758B00758D00D0E0D0D0C295C2DF
:1001100094C293D2AF32C295C294C293206E0D2086
:10012000660A7414D5E0FDE57EF45290758B007577
:100130008D00D0E0D0D0D2AF32758A00D263757C0A
:1001400000C28DD262212C01C4306805206602D223
:100150009501C4306805206602D29401C430680558
:10016000206602D29301C4D29230680A20660774D6
:1001700010D5E0FDD29501C4D29130680A206607FF
:100180007410D5E0FDD29401C4D290D29230680AA6
:100190002066077410D5E0FDD29301C4C2AFC2AD92
:1001A00053E6EFC0D0C0E0D2D3D2AFE57D6009E521
:1001B0007A6005757A004141757A01C2CEE52A6000
:1001C00007207449152A410D7800790020742EE526
:1001D00080307E01F430E70278FF53DACF207E03CF
:1001E00043DA20307E0343DA10C2D8C271E5803092
:1001F0007E01F430E70279FFC3E89970CB306103E8
:10020000752A40207403752A40885FD27020740DCF
:10021000E52B6004152B411D43DA01C2D820700282
:100220004130A85F206102C270207402412E8822F2
:100230007882B60403852224C3E52594404002D287
:100240006420CF0AD0E0D0D043E610D2AD32C2CF86
:10025000053AE57D6009E57B6005757B00612E75DB
:100260007B017802E52A6005307402152AC3E55F38
:1002700094014005756200418A756300756C00E564
:10028000622401F56250037562FF7982B7020D3076
:100290006D1DC3E52294324016854D227982B70345
:1002A0000E306D0BC3E52294324004798E8722C351
:1002B000E523952260084004152341BE0523D8CAD2
:1002C000056CE56C7002156CD56D63756D01780574
:1002D000C3E56C956E4057C3E56C956F5008780187
:1002E000756D030202F2C3E56C95705005780175D7
:1002F0006D01C3E5659524401E7982B70402612330
:10030000206D14852465E56C046003856E6C756D45
:100310000175233C02032EE5652850057565FF61D4
:1003200023F565E5650470067563FF756CFFD0E025
:10033000D0D043E610D2AD32C2AFC0D053E67FC2B8
:1003400060759100855694855795759104D0D0D2EB
:10035000AF32C2AF53E6EFC2ADC0D0C0E0C0F0D202
:10036000D3D2AFA8FBA9FCE57D6007C3E913F9E888
:1003700013F8C2D830710261C453DACF207E034330
:10038000DA10307E0343DA20D271E580307E01F44A
:1003900020E702619B88278928A1A953DACF207E14
:1003A0000343DA20307E0343DA10C2D8C2713074BE
:1003B00002A1957800E580307E01F430E702A19536
:1003C000885FA17D53DACF207E0343DA20307E039D
:1003D00043DA10C271206102819D53DACF207E037F
:1003E00043DA10307E0343DA20C2D8D271885A89AA
:1003F0005BC3E89558F8E99559F97B007E087A00C7
:10040000C3E8948CE994005005755E00818F8821C3
:1004100078A2E6A8216055C3E894C8E99400500882
:10042000E4D2E4FB7A0A816AC3E89468E994015053
:1004300008E4D2E3FB7A0F816AC3E894D0E994021E
:100440005008E4D2E2FB7A1E816AC3E894A0E994E2
:10045000055008E4D2E1FB7A3C816AC3E89498E94C
:1004600094085008E4D2E0FB7A787E00C3E8955CFB
:0F047000FCE9955DFD30E70AECF42401FCEDF4A6
:10047F003400FD755E00C3EC9AED9E5003755E016E
:10048F00885C895D855A58855B597802A17DC3E8E0
:10049F009527F8E99528F9307C02A161307B02A1FC
:1004AF0061307A02A15A20750281C0E9FDE8FC8112
:1004BF00DFE9C313F9E813F8307902A15AE9C3133E
:1004CF00F9E813F8307802A15AE9C313FDE813FCD9
:1004DF0020612CC3EC941CED9402400281F6ED7068
:1004EF001EC3EC94C850180529E52970021529C3BD
:1004FF00E529940A5002A195755F00D270A195E588
:10050F0029600215297400207F037896E624FAFEED
:10051F00E43400FFC3EC9EFCED9FFD50067800799C
:10052F0000A161C3EC94FFED9400400678FF7900C1
:10053F00A161EC8575F0A4C5F0A2F733F8790040FE
:10054F000302057D78FF790002057DE9C313F9E801
:10055F0013F8307C0EE9600278FFC3E81338F8E433
:10056F003400F9C3E894FFE99400400278FF885FF4
:10057F00D270206102A195741FF4552F4BF52FC235
:10058F0074EB7002D274752A40307403752A0A30E6
:10059F006102A1A920740353DAFE207403752B2086
:1005AF00D0F0D0E0D0D0D2AD43E6103279010205C1
:1005BF00D979030205D9790A0205D9791E0205D91D
:1005CF0079640205D979C80205D97817E4D5E0FD19
:1005DF00D8FAD9F6227A147B780206007A107B8C2F
:1005EF000206007A0D7BB40206007A0B7BC8020666
:1005FF00007902B27DE4D291D5E0FDD294D5E0FD31
:10060F00C294D5E0FDC291D5E0FDD295E576D5E057
:10061F00FDC2957496D5E0FDD9D9EAF8D5E0FDD89D
:10062F00FBDBCED29122C37C007D0075F00005F07C
:10063F00EA33FAEB33FB50F6EB13FBEA13FAC3E999
:10064F00FFE8FEE89AF8E99BF95004EFF9EEF8B3EA
:10065F00EC33FCED33FDD5F0DFEDF9ECF822E88952
:10066F00F08A20D2D4F8A9F07B0030F70B7BFFF48F
:10067F002401F8E9F43400F9E88520F0A4ADF0F88E
:10068F00E98520F0A4AFF0FEED2EF974003FFA7C5F
:10069F0004C3EA13FAE913F9E813F8DCF48BF0302A
:1006AF00F70AE8F42401F8E9F43400F9E889F0C214
:1006BF00D4F8A9F0227882B60403020763C3E55F7A
:1006CF009419401EE52D54067018206D3678057963
:1006DF0094E7146007780A1460027812C3E5419812
:1006EF00401F306D09856765756CFF756D0185223B
:1006FF0024E4F545F546F547F548F549C26D02077F
:10070F0063D26D7994E7147013E523F43333F9133F
:10071F00F8E9540104F9E854FE020757E71414707E
:10072F0014E523F4333333F913F8E9540304F9E8E8
:10073F0054FC02075FE523F433333333F913F8E93D
:10074F0054070404F9E854F8C39440F8E99400F905
:10075F008845894622C3E54113F9E54013F8C3E5FF
:10076F004598F8E54699F9500CC3E89480E994FF51
:10077F00401602079BC3E8947FE9940050030207D9
:10078F009B787F790002079B788079FF884A894B95
:10079F0022E54A2547F8E54B3548F9854B20E430EB
:1007AF000701F43549FA30E709C3EA94F04015021E
:1007BF0007D9C3EA940F50030207D978FF79FF7A5C
:1007CF000F0207D9780079007AF0C3E524956450B9
:1007DF000AC374019524500B0207F7E54B20E70E6F
:1007EF000207F7E54B30E706884789488A492278A0
:1007FF00A4E6FAC3E54A33F8E54B33F912066DE97F
:10080F0030E70BC3E89480E994FF40130132C3E84B
:10081F00947FE9940050020132787F790001327899
:10082F008079FFE820E715C3E52398F84009C3E86E
:10083F00940140030208597801020859E8F4240191
:10084F002523F8400302085978FF884C2278A5E643
:10085F00FAA848A94912066DE930E70CC3E89401DC
:0F086F00E994FF401602088EC3E894FFE9940055
:10087E00500302088E78FF790002088E780179FF06
:10088E00E920E715C3E54C98F84009C3E894014008
:10089E00030208B578010208B5E8F42401254CF8E6
:1008AE0040030208B578FF88242278FFC2642069CD
:1008BE003D206A12D264C3E541940A4009C3E5257E
:1008CE0094405002C26479A1E76023E541601F7431
:1008DE00FF8541F0848539F0306A0375F005A4F880
:1008EE00C5F0600278FFC3E895675002A867886676
:1008FE0022C3E54094C8E5419400E56650031421F7
:10090E0010046002F566227883E6F520120FD17589
:10091E00E8901205BB75E890E5E820ECFBA8BDA9B0
:10092E00BE12106F757100757200C3740013FD74E2
:10093E0000606613FC74002CFC74003DFDECFAEDB7
:10094E00FBC3E89AE99B4014E5712400F571E5724A
:10095E003400F572EA2CFAEB3DFB80E5AE71AF7216
:10096E00C3E57213F9E57113F8C3E913F9E813F847
:10097E007A03C3E913F9E813F8DAF7AA201A700913
:10098E007571007572000209A71AEA6008EE28FE5A
:10099E00EF39FFDAF88E718F722275E89022788324
:1009AE00E6FFE5E820ECF7A8BDA9BE0573C3E57325
:1009BE0094084052757300E9FA79A0E76044EA7032
:1009CE0007E574601B0209E2C3E895746010E574D4
:1009DE005006600C140209EE0460F90209EEE5748B
:1009EE00F574C39472401B7564C0C39404401375B0
:1009FE006480C39404400B756440C3940440037533
:100A0E00640075BB0622EFC39401601F7400601B67
:100A1E00C3E894FFE994035012C3E89571E9957207
:100A2E005009E564600C1564020A40E564F4600246
:100A3E000564A864C3E524985002A824C3E895650C
:100A4E00400AA865E565F4600385656488258826F7
:100A5E00E573B4070375BB1022743279A687F0A430
:100A6E00C5F0A2F733F8C3E895644002A864882263
:100A7E008824882588268867227540007541F022D3
:100A8E00C2AF75C820A8CCA9CDAA3A30CF010A753D
:100A9E00C824D2AFC3EA13FAE913F9E813F8AB3B53
:100AAE00AC3C883B893CC3E89BF8E99C20690A541E
:100ABE007FF930670261B1610EAD3D8A3DF9EA9D65
:100ACE00547FFA600478FF79FFAE3EAF3F8B3E8CC9
:100ADE003FC3EC9FFCC3E99CF542A83BA93CC3E88D
:100AEE009EF8E99FF9C3E54113FBE54013FAE82AA6
:100AFE00F540E93BF54150067540FF7541FF6158E1
:100B0E00AA40AB41AC40AD417E047F02C3EB9404DE
:100B1E0040021E1FC3EB940840021E1FC3ED13FDBF
:100B2E00EC13FCDEF7C3EA9CFAEB9DFBEF6009C306
:100B3E00E913F9E813F8DFF7EA28FAEB39FB8A40F4
:100B4E008B4150067BFF8B408B41C3EB94025002CE
:100B5E00D2673069047F0361837892E6FFC3E5377D
:100B6E00948240110FC3E53794A040010FC3EF9458
:100B7E000640027F057E03E541C4540FF9E541C4EA
:100B8E0054F0F8E540C4540F28F8C3E89EFAE994EF
:100B9E0000FB4009C3EA9402EB940050047A02E48D
:100BAE00FB61FDAA40AB41EBC4FEEAC4540F4EFC00
:100BBE00C3EA9CFAEB9400FBC3E813C313F8EA28CC
:100BCE00FAEB3400FB8A408B41C3EB94024002C225
:100BDE00677803EBC4FE7B00EAC4540F4EFAC3EAF7
:100BEE0098FA4005C3940250027A027892E6FF30DA
:100BFE00600261FD855256855357D26043E680C32D
:100C0E00E49AF8E49BF9C3E833F8E933F930670264
:100C1E00819EE8FAE9FBD3E913FDE813FC885289BB
:100C2E0053C3EF94036038EF20E00DE82CF8E93D54
:100C3E00F9ECFAEDFB020C59E828F8E939F9C3E8AA
:100C4E002402F8E93400F97AFE7BFFC3EF940340E7
:100C5E000E8A548B55884E894F8C508D5181D28877
:0F0C6E005489558A4E8B4F8C508D51306920C35D
:100C7D00E53394034019E542A2E713F8E555F42452
:100C8D000138400B20E7087554FFF42401F5558118
:100C9D00D2E8FAD3E813FC8852C3EF94036020EF37
:100CAD0020E007E82CF8ECFA81BEE8282402F87A57
:100CBD00FEC3EF940340088A54884E8C5081D2882D
:100CCD00548A4E8C50E56BC3335002646BF56B3018
:100CDD00600281DC753404D26043E680E52D540654
:100CED00601FA840A941C2AF53E67F759100C3E4D0
:100CFD0098F594E499F595759104D26043E680D208
:100D0D00AF22D265754400752000306B037520400D
:100D1D00020D2ED265754400752040306B03752091
:100D2D0000D2AF7801206722E52D54066002C2651E
:100D3D00C3E5419405401378029405400878039467
:100D4D000540027806306902780A206019E5446092
:100D5D001530690AC3E53394034003D53406D2AF89
:100D6D00D26CC11091E4D2AF0000C2AF20672AE56A
:100D7D0041C3FB940F40027B0FEB2405307301231D
:100D8D00306A02742820620123F93069027982E504
:100D9D008D13E58B13C39940B10544E59B5440B5C4
:100DAD002002A1FA30690A08C3E8940A400108A19B
:100DBD0057206502A12EC26553E67F7591003067FD
:100DCD00107594007595FC759104D26043E680A171
:100DDD002EAE40AF41C3EE33FEEF33FF50047EFF26
:100DED007FFFC3E49EF594E49FF595A1D4C3E5334D
:100DFD0094025002A12E306502A12ED802C10EA17F
:100E0D0057C26C53E67F7591008554948555957541
:100E1D009104854E56854F57D26043E680D2AFE59B
:100E2D002D54066008206A020533020E4A306C0DFF
:100E3D00206B0A206507158115810216B4227800F2
:100E4D003064053065027801E53775F007A4F9E5E2
:100E5D00F028F5F0E9A2F013A2F113A2F213F53781
:100E6D00C394785003753778C3E53795384008D269
:100E7D0066C295C294C293306002C1848550568576
:100E8D005157D26043E68022207D11C2AF754302D7
:100E9D00D291C292D2AF759F1102106CC2AF754341
:100EAD0002D291C290D2AF759F1102106C30724573
:100EBD00207D22C2AF754303900178757E02C293E7
:100ECD00D290D292306204D294C1DAC291D2AF756F
:100EDD009F0102106CC2AF754303900178757E02BD
:100EED00C295D292306204D294C1FAC291D2AF753A
:100EFD009F2102106C207D17C2AF754303900153E3
:100F0D00C293306202D294D2AF759F0102106CC2AF
:100F1D00AF754303900153C295306202D294D2AFA4
:100F2D00759F2102106C207D11C2AF754304D292C2
:100F3D00C290D2AF759F2102106CC2AF754304D21F
:100F4D0090D292C292D2AF759F0102106C30724353
:100F5D00207D20C2AF754305900167757E04C29454
:100F6D00D291306204D295E178C292D2AF759F11C1
:100F7D0002106CC2AF754305900189757E01C29454
:100F8D00D291306204D293E198C290D2AF759F1185
:100F9D0002106C207D17C2AF754305900149C294B4
:100FAD00306202D295D2AF759F1102106CC2AF752F
:100FBD00430590015DC2943062EBD293D2AF759F21
:100FCD001102106C207D13C2AF754306D290D292E0
:100FDD00C291D2AF759F0102106CC2AF754306D29C
:100FED0092C291D2AF759F2102106C307244207D58
:100FFD0020C2AF754301900189757E01C295D292D1
:10100D00306204D2930116C290D2AF759F210210A7
:10101D006CC2AF754301900167757E04C293D29087
:10102D00D292306204D2950138C292D2AF759F012F
:10103D00016C207D16C2AF75430190015DC29530E4
:10104D006202D293D2AF759F21016CC2AF7543017D
:10105D00900149C293306202D295D2AF759F01C201
:0E106D006622900147757E00C295C294C29320
:10107B00D292D291D290C2622278807607087607FC
:10108B000876010876040876FF0876FF08760A08CA
:10109B007602087601087601788C760108760008CE
:1010AB0076B40876FF0876FF0876FF087603087695
:1010BB00FF0876010876FF0876250876D008767843
:1010CB000876C80876040876FF08760108760008CB
:1010DB00767A08760A087601087601087600087693
:1010EB00FF227887E6FFC272BF0302D2727888C2F2
:1010FB007DE630E102D27DC27E7889E630E102D214
:10110B007EC3EF94026008758E01D27302111F75B6
:10111B008E00C273227880E6149000809378A4F638
:10112B007881E6149000809378A5F67886E6149083
:10113B00008D9378A6F6789FE6F8700108C3E894C3
:10114B001140027811E82828F56E256E256E28F5DA
:10115B006F256E2828F570789CE67538FF75390C6D
:10116B00B402067538A075390AB403067538827552
:10117B00390578A3E61490009A93F569116F222232
:10118B007896E6FA7897E6FB7888E6B40305C3EB26
:10119B00940EFB307F047A007BFFC3EB9AFCC39465
:1011AB008250027C827575000575EC8575F0A4C3C1
:1011BB00E5F0947D40F222D27F318B1205CA7A0082
:1011CB007B007C101205C0E55F2AFA74003BFBDC48
:1011DB00F37C04C3EB13FBEA13FADCF7FEC27F319B
:1011EB008B22E5EF20E6037520000520903FFFE5FD
:1011FB0020146006901FFF1460009304600375EFCA
:10120B001253D9BF7581C043FF801205BB75EF0226
:10121B0043B203E5B3240420E70DF521E5E320E019
:10122B00068521B343E301116F7580FF75A400752B
:10123B00F19075D47F75908775A5BF75F2BF75D585
:10124B000075A60175E241E4F8F6D8FD756B011146
:10125B008412170378988676753001C2AF1205D4C5
:10126B001205E41205CA1205EB1205CA1205F21299
:10127B0005CA1218251205D41205D41205CFC2AF18
:10128B0078FA79FA308707D9FBD8F7021C0011EDF1
:10129B003120318A318B78988676116F75A900755C
:1012AB00B680757D0075885075891275C824759147
:1012BB000475D84075A82275B80275E690759B80A9
:1012CB00759D0075D10E75BC5875BB0675BA117539
:1012DB00E8801205BBD2AF12091553DACF207E037B
:1012EB0043DA20307E0343DA1043DA01C2D8C271ED
:1012FB001205D4D2617B037A0CE55E70077A0CDBA6
:10130B00030212891205CA207003021289C270E50A
:10131B005FC3940240E1E52F541F856160F561B511
:10132B0060D5DAD5C26153DACF207E0343DA2030A1
:10133B007E0343DA10C2D8C27178A2E67008D27469
:10134B00E52F54E0F52FC2757529001205CF3074C7
:10135B0009C3E529940A4002D2751205C078023000
:10136B0074027800C3E55F9840F0C2AF1205E41237
:10137B0005E41205E4D2AF1205D4754D001205C079
:10138B00788CE6C39401500302145EE530C39401DC
:10139B00500302145E207435C3E55F94FF500302C3
:1013AB00145EC2AF1205F9D2AF1205CFC3E55F943D
:1013BB000150EFC2AF1205E41205C51205E4D2AF1E
:1013CB001205CFC3E55F94FF40E90218AA7F05D24F
:1013DB007F318B1205CFC2AFC27F318BAE5FC3E5BE
:1013EB005F947FD2AF40761205BBC2AF1205F9D224
:1013FB00AFDFDC31C2C3EE94057897F61205D41239
:10140B00174412182D7F0AD27F318B1205CFC2AF32
:10141B00C27F318BAE5FC3E55F947FD2AF50E612D4
:10142B0005BBC2AF1205E41205C51205E4D2AFDF4E
:10143B00D631C2EE24057896F61205D41217441253
:10144B00185C1205CF318BC3E55F94FF500261A08E
:10145B000218AAC3E55F954D4003855F4D1205CF7A
:0E146B0078017988E7B403027805C3E55F983D
:1014790040026188C2AF1205F91205F91205F9D2C5
:10148900AF1205D4753000E4F531F5320531E53197
:10149900F470390532789AE67819146012783214A2
:1014A900600D787D14600878FA146003753200C302
:1014B900E53298401715327531B478998676C2AFFE
:1014C9001205F9D2AF789886761205CF1205C5E5CF
:1014D9002A7005307402418978012074027806C3A4
:1014E900E55F9840A71205CFE52A7003021289C269
:1014F900AF116FE4F522F523F524F525F526F56AF4
:10150900D2AF7885E6C333F568E4F545F546F54786
:10151900F548F549F573F52CF52DF537757308750B
:10152900BB101205BB1209A8E5E820ECFBA8BDA970
:10153900BEE97001F888741209AC75730875BB109F
:101549007887E6FE760211ED7887EEF6C2AF75640C
:10155900FF120A67852264852265852266D2AF75E6
:10156900220175240175250175260185636C756D48
:101579000175B69075A903757D017888E6B40307EE
:10158900C27D307602D27DD268D269753300120FDE
:10159900D1120FF8120A87120A8E120A87120A8EBE
:1015A900120A870215BBC2AF11EDD2AF7573007570
:1015B900BB06120D201206C4120E4B120E95120A0A
:1015C9008E120D0F306D031207642067031208B8DD
:1015D9003067031208FF120E4B120EBA120A8E124E
:1015E9000D20306D031207A0120E4B120F33120A91
:1015F9008E120D0F306D031207FE120E4B120F5A89
:10160900120A8E120D20306D0312085C120E4B1255
:101619000FD1120A8E1209A8120D0F120E4B120FBA
:10162900F81209AC120A8E30692F206B2C85676479
:1016390085676585636C756D0179187A0CC3E53327
:10164900994009C269D26A8A35021662C3E55F9474
:101659000140030215BB0216BC306A1B206B18E55A
:1016690035147004C26AA1AFF535C3E55F94014032
:10167900030215BB0216BC753600C3E5629401402E
:101689000985676585636C756D01C3E56278FA98AC
:101699005021307404E52A601A78F0306B058567AB
:1016A900647820C3E541985002A1BB0536E55F6027
:1016B90002C1BF753600C2AF116F7887E6FE7602A8
:1016C90011ED7887EEF6E4F522F523F524F525F5F5
:1016D90026F568C26875A90075B680757D00D2AF18
:1016E9001205BB116F307406E52A70024189788DA5
:1016F900E6C39401400261658190901A0D78201229
:101709001786E520B4A50CA3121786E520B45A0361
:101719000217241184121744021743901A03788080
:101729007B0A121786A308DBF9901A0F788C7B18AD
:10173900121786A308DBF9901A2722C2AF1217C520
:1017490012179F901A00740E12178BA374041217A4
:101759008BA3741412178B901A0378807B0A1217C3
:101769008AA308DBF9901A0F788C7B1812178AA3C1
:1017790008DBF91217D81217B6901A2722E493F644
:1017890022E6438F01538FFD75EF0275B7A575B733
:10179900F1F0538FFE22438F02438F0175EF0275DB
:1017A900B7A575B7F1901A0DF0538FFC22901A0D59
:1017B90074A5F18B901A0E745AF18B227A3079D074
:1017C9007820901A40F186E520F709A3DAF7227A02
:1017D9003079D0901A40E7F18B09A3DAF922AB7777
:1017E900A878BB01027980BB02027981BB03027927
:1017F90082BB04027994BB05027983BB0602798610
:10180900BB07027992BB08027987BB0902799CBBA5
:101819000A027988BB0B027989E8F7227C0512054F
:10182900D4DCFB22C2AF1205E41205EB1205F21259
:1018390005F91205C51205E41205EB1205F21205A8
:10184900F91205C51205E41205EB1205F21205F9A4
:10185900D2AF22C2AF1205F91205F21205EB120539
:0D186900E41205C51205F91205F21205EB97
:101876001205E41205C51205F91205F21205EB125E
:1018860005E4D2AF22AE77AF78C2AF1205E41205F7
:10189600E41205E41205C5DEF21205F91205C5DFEC
:1018A600F8D2AF22112D1125112575770175780112
:1018B600757900118B7C05AD5F1205D4C3ED955F7C
:1018C60070F5C3E55F9401400AC3E55F94FF4034B9
:1018D6000218E81217E7121744112DC2AF75EF125E
:1018E6001125DCD30579C3E5799403500280C41130
:1018F600250578E5771490009F93F808C3E5789856
:10190600500280AC112511250577C3E577940C505C
:1019160002809A121084121744C2AF75EF12112575
:0319FD000211EDE7
:101A00000E041407070104FFFF0A020101A55A0191
:101A100000B4FFFFFF03FF01FF25D078C804FF01DA
:081A200000FF0A010100FFFFB5
:101A4000234F76736B794D5232304150726F2320A1
:101A500023424C48454C492346333930232020202B
:101A60002020202020202020202020202020202076
:101C0000C2AFC2D353D9BF7581C043B20343FF8073
:101C1000752438752503B1C975EF0275E24043F1AB
:101C20008053A47F75D400D2877DFA780379E67C4F
:101C300010752200752300901DD67B0675249875BB
:101C400025013087028142208708D8FBD9F9DCF7CB
:101C500081B4308708D8FBD9F9DCF781B4B189E4C5
:101C600093A3C39A6004DDC381B4DBDBB17B600264
:101C7000812B7B08E493FAA3B15CDBF87A30B15C8A
:101C8000752200752300B17BEAFCEBFDC3ED94FEE9
:101C9000400EB17B8A278B28ED30E0048A828B834B
:101CA000B17B7AC270D8C3ED94FE601350CEBD00F4
:101CB00025EC60097520007521FF0200008100A855
:101CC00027A9280809D804D90281D3B17FEA89AAB3
:101CD000F281C50D81A0C3ED94035049EDA2E092BD
:101CE000007AC5C3E5829400E583941C50902000DF
:101CF00010438F02438F0175B7A575B7F1F030001F
:101D00001FA827A9280809438F01538FFDD804D99C
:101D100002A12089AAE275B7A575B7F1F0A3A10DBC
:101D2000538FFC817C7AC1BD030CE493A3FAB140CC
:101D3000DCF8B138817C817EAA22AB23B15CEBFA5E
:101D4000EA6222752608C3E52313F523E52213F57D
:101D50002250066323A0632201D526EAB1C9B1C986
:101D600075260AEAF4200102D287300102C287B147
:101D7000C9C3134002C201D526EB22B17FEAFB2082
:101D80008702A17F308702A184752608AE24AF2583
:101D9000C3EF13FFEE13FEB1CDB1C9C3EA13308711
:101DA000024480FA30E703632201C3E52313F523DD
:101DB000E52213F52250066323A0632201D526D91C
:101DC000E52265236523F52222AE24AF250E0FDE22
:101DD000FEDFFCD20122424C48656C693437316326
:041DE000F390060175
:00000001FF
